:0200000001A558
:0D000B00301617D8058690780C328690329A
:02001B008178EA
:1000230081A1D5253D7525B4C0D0C0E0A29230177B
:1000330001B3500BD2011165D0E0D0D00200BBD583
:100043001812E519601D15197518FF300806E51912
:100053007002C2B2300A07D50B04050AC212D0E0FF
:10006300D0D032C28CC205051ED2B780F17588008C
:10007300759850758BF4758DF4758C00758A0075C1
:10008300892275885022758800758CC0758AC07561
:100093008D00758B00758922750E037588507598D0
:1000A30000227590F775B07775D01075815F7587ED
:1000B300807525B41170F15FC2AF75200075210002
:1000C300752200A2929217F11A740020170274800D
:1000D3001207EC1207C1F521C20DC20CC2B21207FE
:1000E3007F100171200B02215875815F111775A8CC
:1000F30090780079007A00DAFED9FAD8F6F12AC2AC
:10010300AF510DC2AF1117751E00E51E60087519BA
:10011300007518648014740120170274811207ECAF
:100123001207C1F5191207C1F518750A00D2051196
:1001330070D212C211750B64200B0830070530080A
:1001430002D2B275A88230120A200D04A2B692B769
:100153002005F3D2B775815FC2AF11171170C202C8
:10016300C207C203C2B2750E0A300B02210075A882
:1001730092200D04A2B692B73002F6D2B730090826
:100183003007AC20030280F5300A1BC2AF30111BCD
:10019300740820170274881207EC1207C1C50AB548
:1001A3000A00C50A400502010221322005FB74033F
:1001B30020170274831207EC1207C1FD1207C1FA5C
:1001C3001207C1FBB523005025E5238AF0B5F000E3
:1001D30050D4EAC395238DF0A4AEF0FFEAC39B315C
:1001E300F404F5F0E51EB5F00050BB02010DED80FF
:1001F300F0F42401CE7D0950042ED380042E400157
:100203009ECF33CF33DDF013CF22C205200D0A7901
:1002130000A2B692B750F5D9F8D2B7740A201702E4
:10022300748A1207EC1207C1F51E300602151E125E
:1002330007C1F51FF1717519FF7518FF9117740F39
:10024300201702748F1207EC1207C1FB74102017DA
:100253000274901207EC74A11207FD1189780C75D2
:10026300A88AC2B3D293D216D2D5300702C2B751ED
:10027300DEDBFC90098951F4AD1E71197926E75133
:10028300FE09E9B51DF8200606AD1F7119151CE519
:100293001851FEE51951FE51DE51DE1207C9C2AFF6
:1002A300C293C216D2B7D2B3C2067590F7E51C60EB
:1002B300020170F11A740920170274891207EC12F3
:1002C30007C11207EC79261207C16004F70980F70A
:1002D300891D7819120849D206410DB2D57A07C291
:1002E300003000FDDAF9B2D5C2003000FD751A0501
:1002F30022E493600551FEA380F7227A08C31350CA
:1003030008C2003000FDD51A0AB2D5C2003000FD84
:10031300751A05DAE8227A08D2B5000030B5FD0077
:10032300A2B4500AC200C2B53000FDD51A0CB2D532
:10033300C200C2B53000FD751A05DADCC2B4D2B50D
:10034300000030B5FDC2B5D2B4DDCB22E4F50CF527
:100353000D790EE501B42D01221986F018E618DA9D
:100363000474007A0171EBF7DAEFE50D250DD4F58E
:1003730000E50C350CD4F501E43400D4F502E500B6
:10038300250DD4F500E501350CD4F501E502340063
:0E039300D4F5028500038501048502057C0473
:1003A100C3E50513F505E50413F504E50313F503AA
:1003B100DCEEE5002503D4F500E5013504D4F501B3
:1003C100E5023505D4F502A91D1919E50071D9E534
:1003D1000171D9E50271D922F5F0540F4430F719B2
:1003E100E5F0C4540F4430F71922540F53F00FC4F1
:1003F10045F022A2E092F7A2E192F6A2E292F5A2E2
:10040100E392F4A2E492F3A2E592F2A2E692F1A2BF
:10041100E792F0E5F022900989E49360059157A3F2
:1004210080F7741020170274901207ECAD1E1207AA
:10043100C171F49157DDF77926E7915709E9B51DA7
:10044100F820060BAD1F1207C171F49157DDF76358
:1004510019FF6318FF227A08FBC3E51913F519E5A3
:100461001813F518EB30E001B3500663180863194F
:1004710084EB03FBDAE322D50E111117750E03D2BB
:100481000020D504758CDD32758CC0327B007C0078
:10049100209805DCFBDBF722E599C29822C299324C
:1004A1003098FAE599C298B42402A1B2B43EEE752F
:1004B100993E3099FDC299918DB4300B9008E67543
:1004C1008CC0758AC0800CB4313C9008FD758CDD00
:1004D100758ADDF162F171C298C2B3C205D293D2BD
:1004E10016C2AF111775880075892275885075A8D5
:1004F100823098FDC293C216D2B37590F711703055
:100501000B0201EC2158B4322C900914F162F17103
:10051100C2B3C205D293D2161189C2AF1117780C9A
:1005210075A88AD2D5C200300004B2D580F720B0B8
:10053100F6C2AF81F5B43327900932F162C2AF112F
:1005410017C2987903C2B712084512084512084527
:10055100B2B7D9F3A2B692B73098F9D2B781F5B450
:10056100520302084EB45604F15F819EB457FB0258
:100571000862300936300733B44730918DB4472BC8
:10058100918DB44126918DA91D90097FF10E7A05B7
:10059100D1FADAFC918DB43002800ED1FAD1FAD1C0
:1005A100FA78007A00F103714FD203918DB40AFBFE
:1005B10032918DB447F5918DB450F0918DB452B212
:1005C100918DB44DE6918DB443E1D1FA7926300C89
:1005D100077A06D1F0776809D1FA918DB45609D519
:1005E1000E04F109D202A1ACB441C0D1FA7A07D10B
:1005F100F0D1FA7A01D1F0F14BD1FA1207C1F70922
:100601007A08D1F0D1FA7A01D1F0F155D1FA120775
:10061100C1F7097B027A03773009DAFB772F09DB0F
:10062100F4891D7A007800F103A91D1919BA000394
:10063100E48034E6F71819DAFA300A2DE51DC3947F
:1006410004F9E7540FFC09E7540FFB09E7540FFACB
:10065100EC75F064A4FCE5F0700B75F00AEBA4FBFB
:100661002AC32C500274FFF5237A007800F103E5C8
:100671001DC39406F9BA00028006E6F71819DAFAE2
:10068100300A617401B52300505AE51DC39408F97D
:10069100E7540FFC09E7540FFB09E7540FC3133468
:1006A10000FAEC75F032A4FC75F005EBA4FB2AC34B
:1006B1002CFC8524F0B5F0005002C5F0C395F0F58F
:1006C1000F8C24740620170274861207EC1207C1DE
:1006D100FA1207C1FB8523F084C33A500274FFB5B7
:1006E1000F009211200902151DD202D207A1AC916F
:1006F1008DF709DAFA22B42E06918DB42CFB22086B
:10070100F60A918DB42CEF2290096B7926E493605F
:0E07110005F709A380F7891D22740C2017023A
:10071F00748C1207EC1207C1F51C2274EE1207EC51
:10072F0079267A121207C1F709DAF9F14B1207C1CC
:10073F00F52EF1551207C1F709891D22740E2017E6
:10074F0002748E0207EC740D201702748D0207ECF1
:10075F00900991E493600AF5993099FDC299A380AD
:10076F00F2229008CA7800E493F6A308B80CF82296
:10077F007902C2B7120845120845120845D2B7C20E
:10078F00B3120845120845120845D2B3D9E4D2B7BF
:10079F00120845301704C2B78002C2B3780A120894
:1007AF0049D2B7D2B322C2B4D2B5000030B5FDD210
:1007BF00B42274A11207FD2004207C08D2B50000DA
:1007CF0030B5FD00A2B433C2B500DCF0D2B4D2B55F
:1007DF00000030B5FD00C2B5D2B480CAE4F51B7479
:1007EF00A01207FD200405E51B12080A80B8C204F9
:1007FF0030B52C30B429C2B400C2B57C083392B4E2
:10080F00D2B5000030B5FDC2B5DCF2D2B4D2B5001E
:10081F000030B5FD30B402D204C2B520040922D293
:10082F000490094B0207629009570207627C14E497
:10083F001470FDDCFA227C0080F51145D8FC2212E1
:10084F0007EB78001207C1F5993099FDC299D8F4DA
:10085F0002049E782612048DF608B82FF8782774B4
:10086F00A01207FD2004ECE526110AE6110A120773
:10087F00B5113C080526B82FE60204B0C0E0C4113C
:10088F0092D0E0540FB40A00400224072430F599A7
:10089F003099FDC2992275990D3099FDC2997599BC
:1008AF000A3099FDC29922C2997599543099FDC2A7
:1008BF00997599583099FDC29980DB9FCFEFFFEF63
:1008CF00CF9F6F4F3F4F6F9FBFDFEFFFEFDFBF9F99
:1008DF007F5F4F3F4F5F7F5472616E736D697474AA
:1008EF00696E67203132303020487A0D0A00547219
:1008FF00616E736D697474696E67203232303020A7
:10090F00487A0D0A005472616E736D697474696E62
:10091F00672031323030202F203232303020487A69
:10092F000D0A00436865636B696E6720525820613A
:10093F007564696F6C6576656C0D0A0049324320EA
:10094F006572726F720D0A004E6F2041434B206625
:10095F00726F6D20736C6176650D0A003030303028
:10096F002E30304E5C303030302E3030572E2F003E
:10097F00413D3030303030302F0082A0B4626060A3
:10098F0060004F5A34485A2020415052532054721D
:10099F0061636B6572207769746820383043343037
:1009AF00353120444A374F4F2076657273696F6E29
:1009BF00202876657220312E3120303720303520B7
:0609CF003137290D0A007A
:00000001FF
